gpasm-2.1.3 (Mar 12 2018)    MC32P7311io.asm    2018-5-14  10:58:41          PAGE  1


LOC  OBJECT CODE     LINE SOURCE TEXT
  VALUE

                      00001 #include "mc32p7311.inc"
                      00001                 LIST
                      00002 ;mc32p7311.inc    Standard Header File, Version 1.00 by Sinomcu
                      00625                 LIST
                      00002 
                      00003         org     0x00
0000   A000           00004         goto    start
                      00005     
                      00006         
0001                  00007 start:      
0001   3CFF           00008         movai      0xff;P1output
0002   5795           00009         movra      OEP1        
0003   3CEF           00010         movai      0xef;P0output
0004   5791           00011         movra      OEP0
0005   3CFF           00012         movai      0xff;P1口数据全1
0006   5794           00013         movra      IOP1
0007   3C01           00014         movai       0x01
0008   5788           00015         movra       MCR         ;外部中断0 下降沿中断
0009   3C00           00016         movai       0x00
000A   57AC           00017         movra       PWMCR0
000B   3C90           00018         movai       0x90
000C   57B1           00019         movra       ADCR1      ;AD采样频率FHIRC/32=1MHz  ,内部参考2V                
000D   3C09           00020         movai       0x09
000E   57B0           00021         movra       ADCR0 ;测内参2V时要开AD              
                      00022         
000F   CF98           00023         bset      TC0EN
0010   CD98           00024         bset      PWM0OE
                      00025         
0011   CFAC           00026         bset      PWMCR0,7   ; 允许PWM1 翻转输出到PWM0 故PWM0无需设置
                      00027         
0012   CF9C           00028         bset      TC1EN
0013   CD9C           00029         bset      PWM1OE
0014   3C95           00030         movai     0x95
0015   578C           00031         movra     DRVCR   ;增强驱动能力选择                        
                      00032         
0016                  00033 LOOP:         
0016   7390           00034          COMR   IOP0      ;测试32M 时，io翻转频率1M 即为准确值
0017   0000           00035          NOP
0018   A000           00036          GOTO   LOOP     
                      00037          
                      00038          END
gpasm-2.1.3 (Mar 12 2018)    MC32P7311io.asm    2018-5-14  10:58:41          PAGE  2


SYMBOL TABLE
  LABEL                             VALUE

ADCR0                             000001B0
ADCR1                             000001B1
ADCR2                             000001B2
ADRH                              000001B4
ADRL                              000001B5
ANSEL0                            000001B6
ANSEL1                            000001B7
DRVCR                             0000018C
FSR0                              00000184
FSR1                              00000185
HIBYTE                            00000183
INDF0                             00000180
INDF1                             00000181
INDF2                             00000182
INDF3                             00000189
INTE                              0000018A
INTF                              0000018B
IOP0                              00000190
IOP1                              00000194
KBCR                              0000018E
LOOP                              00000016
LVDCR                             000001AF
MCR                               00000188
OEP0                              00000191
OEP1                              00000195
OSCCALH                           000001FB
OSCCALL                           000001FC
OSCM                              000001AE
PCL                               00000186
PDP0                              00000193
PDP1                              00000197
PFLAG                             00000187
PUP0                              00000192
PUP1                              00000196
PWM0DE                            000001A8
PWM1DE                            000001A9
PWM2DE                            000001AA
PWMCR0                            000001AC
PWMCR1                            000001AD
T0CNT                             00000199
T0CR                              00000198
T0DATA                            0000019B
T0LOAD                            0000019A
T1CNT                             0000019D
T1CR                              0000019C
T1DATA                            0000019F
T1LOAD                            0000019E
T2CNT                             000001A1
T2CR                              000001A0
T2DATA                            000001A3
T2LOAD                            000001A2
T3CNT                             000001A5
T3CR                              000001A4
T3LOAD                            000001A6
_CONFIG0                          00008000
_CONFIG1                          00008001
__32P7311                         00000001
start                             00000001
ADCHS0                            ADCR0,4
ADCHS1                            ADCR0,5
ADCHS2                            ADCR0,6
ADCHS3                            ADCR0,7
ADCKS0                            ADCR1,5
ADCKS1                            ADCR1,6
ADCKS2                            ADCR1,7
ADEOC                             ADCR0,1
ADIE                              INTE,6
ADIF                              INTF,6
ADLEN                             ADCR0,3
ADON                              ADCR0,0
ADR0                              ADRL,0
ADR1                              ADRL,1
ADR10                             ADRH,6
ADR11                             ADRH,7
ADR2                              ADRL,2
ADR3                              ADRL,3
ADR4                              ADRH,0
ADR5                              ADRH,1
ADR6                              ADRH,2
ADR7                              ADRH,3
ADR8                              ADRH,4
ADR9                              ADRH,5
ADSMP0                            ADCR2,0
ADSMP1                            ADCR2,1
ADSMP2                            ADCR2,2
ADSMP3                            ADCR2,3
ADTST                             ADCR1,4
BUZ0OE                            T0CR,5
BUZ1OE                            T1CR,5
BUZ2OE                            T2CR,5
C                                 PFLAG,0
CLKS                              OSCM,2
DC                                PFLAG,1
DRVS                              DRVCR,7
FPWM1INV                          PWMCR0,5
FPWMEN                            PWMCR0,7
FPWMF0                            PWMCR0,0
FPWMF1                            PWMCR0,1
FPWMR0                            PWMCR0,2
FPWMR1                            PWMCR0,3
FSR00                             FSR0,0
FSR01                             FSR0,1
FSR02                             FSR0,2
FSR03                             FSR0,3
FSR04                             FSR0,4
FSR05                             FSR0,5
FSR06                             FSR0,6
FSR07                             FSR0,7
FSR10                             FSR1,0
FSR11                             FSR1,1
FSR12                             FSR1,2
FSR13                             FSR1,3
FSR14                             FSR1,4
FSR15                             FSR1,5
FSR16                             FSR1,6
FSR17                             FSR1,7
GIE                               MCR,7
HFEN                              OSCM,0
HIBYTE0                           HIBYTE,0
HIBYTE1                           HIBYTE,1
HIBYTE2                           HIBYTE,2
HIBYTE3                           HIBYTE,3
HIBYTE4                           HIBYTE,4
HIBYTE5                           HIBYTE,5
HIBYTE6                           HIBYTE,6
HIBYTE7                           HIBYTE,7
INDF00                            INDF0,0
INDF01                            INDF0,1
INDF02                            INDF0,2
INDF03                            INDF0,3
INDF04                            INDF0,4
INDF05                            INDF0,5
INDF06                            INDF0,6
INDF07                            INDF0,7
INDF10                            INDF1,0
INDF11                            INDF1,1
INDF12                            INDF1,2
INDF13                            INDF1,3
INDF14                            INDF1,4
INDF15                            INDF1,5
INDF16                            INDF1,6
INDF17                            INDF1,7
INDF20                            INDF2,0
INDF21                            INDF2,1
INDF22                            INDF2,2
INDF23                            INDF2,3
INDF24                            INDF2,4
INDF25                            INDF2,5
INDF26                            INDF2,6
INDF27                            INDF2,7
INDF30                            INDF3,0
INDF31                            INDF3,1
INDF32                            INDF3,2
INDF33                            INDF3,3
INDF34                            INDF3,4
INDF35                            INDF3,5
INDF36                            INDF3,6
INDF37                            INDF3,7
INT0IE                            INTE,2
INT0IF                            INTF,2
INT1IE                            INTE,3
INT1IF                            INTF,3
KBCR0                             KBCR,0
KBCR1                             KBCR,1
KBCR2                             KBCR,2
KBCR3                             KBCR,3
KBCR4                             KBCR,4
KBCR5                             KBCR,5
KBCR6                             KBCR,6
KBCR7                             KBCR,7
KBIE                              INTE,4
KBIF                              INTF,4
LDRVS                             DRVCR,6
LFEN                              OSCM,1
LVDEN                             LVDCR,7
LVDF                              LVDCR,0
LVDS0                             LVDCR,3
LVDS1                             LVDCR,4
LVDS2                             LVDCR,5
LVDS3                             LVDCR,6
MINT00                            MCR,0
MINT01                            MCR,1
MINT10                            MCR,2
MINT11                            MCR,3
OSCCAL0                           OSCCALL,0
OSCCAL1                           OSCCALL,1
OSCCAL10                          OSCCALH,2
OSCCAL2                           OSCCALL,2
OSCCAL3                           OSCCALL,3
OSCCAL4                           OSCCALL,4
OSCCAL5                           OSCCALL,5
OSCCAL6                           OSCCALL,6
OSCCAL7                           OSCCALL,7
OSCCAL8                           OSCCALH,0
OSCCAL9                           OSCCALH,1
P00ANS                            ANSEL0,0
P00D                              IOP0,0
P00OE                             OEP0,0
P00PD                             PDP0,0
P00PU                             PUP0,0
P01D                              IOP0,1
P01OE                             OEP0,1
P01PD                             PDP0,1
P01PU                             PUP0,1
P02ANS                            ANSEL0,1
P02D                              IOP0,2
P02OE                             OEP0,2
P02PD                             PDP0,2
P02PU                             PUP0,2
P03ANS                            ANSEL0,2
P03D                              IOP0,3
P03OE                             OEP0,3
P03PD                             PDP0,3
P03PU                             PUP0,3
P04ANS                            ANSEL0,3
P04D                              IOP0,4
P04OE                             OEP0,4
P04PD                             PDP0,4
P04PU                             PUP0,4
P05ANS                            ANSEL0,4
P05D                              IOP0,5
P05OE                             OEP0,5
P05PD                             PDP0,5
P05PU                             PUP0,5
P10ANS                            ANSEL0,5
P10D                              IOP1,0
P10OE                             OEP1,0
P10PD                             PDP1,0
P10PU                             PUP1,0
P11ANS                            ANSEL0,6
P11D                              IOP1,1
P11OE                             OEP1,1
P11PD                             PDP1,1
P11PU                             PUP1,1
P12ANS                            ANSEL0,7
P12D                              IOP1,2
P12OE                             OEP1,2
P12PD                             PDP1,2
P12PU                             PUP1,2
P13D                              IOP1,3
P13OE                             OEP1,3
P13PD                             PDP1,3
P13PU                             PUP1,3
P14ANS                            ANSEL1,0
P14D                              IOP1,4
P14OE                             OEP1,4
P14PD                             PDP1,4
P14PU                             PUP1,4
P15ANS                            ANSEL1,1
P15D                              IOP1,5
P15OE                             OEP1,5
P15PD                             PDP1,5
P15PU                             PUP1,5
P16D                              IOP1,6
P16OE                             OEP1,6
P16PD                             PDP1,6
P16PU                             PUP1,6
P17D                              IOP1,7
P17OE                             OEP1,7
P17PD                             PDP1,7
P17PU                             PUP1,7
PC0                               PCL,0
PC1                               PCL,1
PC2                               PCL,2
PC3                               PCL,3
PC4                               PCL,4
PC5                               PCL,5
PC6                               PCL,6
PC7                               PCL,7
PD                                MCR,4
PDLYS0                            DRVCR,2
PDLYS1                            DRVCR,3
PDRVS0                            DRVCR,4
PDRVS1                            DRVCR,5
PMODE0                            PWMCR1,0
PMODE1                            PWMCR1,1
PMODE2                            PWMCR1,2
PSPDS0                            DRVCR,0
PSPDS1                            DRVCR,1
PWM0DE0                           PWM0DE,0
PWM0DE1                           PWM0DE,1
PWM0DE2                           PWM0DE,2
PWM0INV                           PWMCR0,4
PWM0OE                            T0CR,6
PWM1DE0                           PWM1DE,0
PWM1DE1                           PWM1DE,1
PWM1DE2                           PWM1DE,2
PWM1OE                            T1CR,6
PWM2DE0                           PWM2DE,0
PWM2DE1                           PWM2DE,1
PWM2DE2                           PWM2DE,2
PWM2INV                           PWMCR0,6
PWM2OE                            T2CR,6
RESS0                             ADCR1,3
STBH                              OSCM,4
STBL                              OSCM,5
T0C0                              T0CNT,0
T0C1                              T0CNT,1
T0C2                              T0CNT,2
T0C3                              T0CNT,3
T0C4                              T0CNT,4
T0C5                              T0CNT,5
T0C6                              T0CNT,6
T0C7                              T0CNT,7
T0DATA0                           T0DATA,0
T0DATA1                           T0DATA,1
T0DATA2                           T0DATA,2
T0DATA3                           T0DATA,3
T0DATA4                           T0DATA,4
T0DATA5                           T0DATA,5
T0DATA6                           T0DATA,6
T0DATA7                           T0DATA,7
T0IE                              INTE,0
T0IF                              INTF,0
T0LOAD0                           T0LOAD,0
T0LOAD1                           T0LOAD,1
T0LOAD2                           T0LOAD,2
T0LOAD3                           T0LOAD,3
T0LOAD4                           T0LOAD,4
T0LOAD5                           T0LOAD,5
T0LOAD6                           T0LOAD,6
T0LOAD7                           T0LOAD,7
T0PR0                             T0CR,0
T0PR1                             T0CR,1
T0PR2                             T0CR,2
T0PTS0                            T0CR,3
T0PTS1                            T0CR,4
T1C0                              T1CNT,0
T1C1                              T1CNT,1
T1C2                              T1CNT,2
T1C3                              T1CNT,3
T1C4                              T1CNT,4
T1C5                              T1CNT,5
T1C6                              T1CNT,6
T1C7                              T1CNT,7
T1DATA0                           T1DATA,0
T1DATA1                           T1DATA,1
T1DATA2                           T1DATA,2
T1DATA3                           T1DATA,3
T1DATA4                           T1DATA,4
T1DATA5                           T1DATA,5
T1DATA6                           T1DATA,6
T1DATA7                           T1DATA,7
T1IE                              INTE,1
T1IF                              INTF,1
T1LOAD0                           T1LOAD,0
T1LOAD1                           T1LOAD,1
T1LOAD2                           T1LOAD,2
T1LOAD3                           T1LOAD,3
T1LOAD4                           T1LOAD,4
T1LOAD5                           T1LOAD,5
T1LOAD6                           T1LOAD,6
T1LOAD7                           T1LOAD,7
T1PR0                             T1CR,0
T1PR1                             T1CR,1
T1PR2                             T1CR,2
T1PTS0                            T1CR,3
T1PTS1                            T1CR,4
T2C0                              T2CNT,0
T2C1                              T2CNT,1
T2C2                              T2CNT,2
T2C3                              T2CNT,3
T2C4                              T2CNT,4
T2C5                              T2CNT,5
T2C6                              T2CNT,6
T2C7                              T2CNT,7
T2DATA0                           T2DATA,0
T2DATA1                           T2DATA,1
T2DATA2                           T2DATA,2
T2DATA3                           T2DATA,3
T2DATA4                           T2DATA,4
T2DATA5                           T2DATA,5
T2DATA6                           T2DATA,6
T2DATA7                           T2DATA,7
T2IE                              INTE,5
T2IF                              INTF,5
T2LOAD0                           T2LOAD,0
T2LOAD1                           T2LOAD,1
T2LOAD2                           T2LOAD,2
T2LOAD3                           T2LOAD,3
T2LOAD4                           T2LOAD,4
T2LOAD5                           T2LOAD,5
T2LOAD6                           T2LOAD,6
T2LOAD7                           T2LOAD,7
T2PR0                             T2CR,0
T2PR1                             T2CR,1
T2PR2                             T2CR,2
T2PTS0                            T2CR,3
T2PTS1                            T2CR,4
T3C0                              T3CNT,0
T3C1                              T3CNT,1
T3C2                              T3CNT,2
T3C3                              T3CNT,3
T3C4                              T3CNT,4
T3C5                              T3CNT,5
T3C6                              T3CNT,6
T3C7                              T3CNT,7
T3IE                              INTE,7
T3IF                              INTF,7
T3LOAD0                           T3LOAD,0
T3LOAD1                           T3LOAD,1
T3LOAD2                           T3LOAD,2
T3LOAD3                           T3LOAD,3
T3LOAD4                           T3LOAD,4
T3LOAD5                           T3LOAD,5
T3LOAD6                           T3LOAD,6
T3LOAD7                           T3LOAD,7
T3PR0                             T3CR,0
T3PR1                             T3CR,1
T3PR2                             T3CR,2
T3PTS0                            T3CR,3
T3PTS1                            T3CR,4
TC0EN                             T0CR,7
TC1EN                             T1CR,7
TC2EN                             T2CR,7
TC3EN                             T3CR,7
TMRCKS0                           PWMCR1,3
TMRCKS1                           PWMCR1,4
TO                                MCR,5
VRS0                              ADCR1,0
VRS1                              ADCR1,1
VRS2                              ADCR1,2
Z                                 PFLAG,2

Errors   :     0
Warnings :     0 reported,     0 suppressed
Messages :     0 reported,     0 suppressed

